:100000000EC015C014C013C012C011C010C00FC064
:100010000EC00DC00CC00BC00AC009C008C011241E
:100020001FBECFE5D1E0DEBFCDBF7CD0ECC0E8CFB6
:10003000FC018081562F5095852380838CEC90E0C5
:100040000197F1F7242F332727FD309520FF03C0B8
:100050008081862B02C08081852380838CEC90E098
:100060000197F1F721FF03C08081862B02C08081B8
:10007000852380838CEC90E00197F1F722FF03C089
:100080008081862B02C08081852380838CEC90E068
:100090000197F1F723FF03C08081862B02C0808186
:1000A000852380838CEC90E00197F1F724FF03C057
:1000B0008081862B02C08081852380838CEC90E038
:1000C0000197F1F725FF03C08081862B02C0808154
:1000D000852380838CEC90E00197F1F726FF03C025
:1000E0008081862B02C08081852380838CEC90E008
:1000F0000197F1F747FF04C08081862B808303C0FE
:100100008081582350832CEC30E0C9010197F1F72E
:100110008081862B8083C9010197F1F7C90101977E
:10012000F1F70895EF92FF920F931F93CF93DF9310
:1001300080E886BD16BCC29ABA9AC39ABB9A82E07E
:1001400087B987E886B9C0E0D0E0EE24FF2420E03C
:1001500000E21EE4C39A369A3699FECF84B195B177
:10016000E80EF91EC398369A3699FECF84B195B140
:10017000C80FD91F2F5F243669F788E390E064E049
:1001800041E056DFC8010197F1F788E390E064E0B1
:1001900042E04EDFC8010197F1F788E390E064E0A8
:1001A00043E046DFC8010197F1F788E390E064E09F
:1001B00044E03EDFC8010197F1F788E390E064E096
:1001C0004C2F36DFC8010197F1F788E390E064E037
:1001D0004D2F2EDFC8010197F1F788E390E064E02E
:1001E0004E2D26DFC8010197F1F788E390E064E027
:1001F0004F2D1EDFC8010197F1F720E0EE24FF2408
:0A020000C0E0D0E0A7CFF894FFCFD4
:00000001FF
